:020000040800F2
:10000000E0020020D9000008B50C00085D060008D9
:1000100000000000000000000000000000000000E0
:10002000000000000000000000000000810F000838
:100030000000000000000000090D00082910000861
:10004000EB00000800000000EB000008EB000008D7
:10005000EB000008EB000008EB000008EB000008D4
:10006000EB000008EB000008EB000008EB000008C4
:1000700061020008EB000008EB000008891000088E
:1000800000000000B51000080000000000000000A3
:1000900000000000EB000008EB000008EB00000887
:1000A00000000000EB00000800000000EB0000086A
:1000B0000000000000000000000000000000000040
:1000C0000448854600F06EF800480047C51800084F
:1000D000C046C046E002002004488047044800476C
:1000E000FEE7FEE7FEE7FEE7FEE7FEE72D1000086D
:1000F000C100000830B50B46014600202022012433
:1001000009E00D46D5409D4205D31D469540491B4B
:100110002546954040191546521E002DF1DC30BD94
:10012000D2B201E00270401C491EFBD2704700228F
:10013000F6E710B513460A4604461946FFF7F0FFE6
:10014000204610BDF0B51FB40646002082B005461B
:100150004024019100901BE0019922460F46304651
:1001600000F042F8049A059B801A994110D310467A
:100170001946224600F028F8361A8F410197224688
:1001800001200021009F00F01FF838184D41009019
:100190002046641E0028DFDC019B00982946324679
:1001A00007B0F0BD064C0125064E05E0E36807CC1C
:1001B0002B430C3C98471034B442F7D3FFF784FF2D
:1001C00080230008A023000810B5202A04DB014684
:1001D000203A9140002010BD914020239C1A0346F4
:1001E000E3401943904010BD10B5202A04DB0846B7
:1001F000203AD040002110BD0B46D340D0402024EF
:10020000A21A91400843194610BD70B58C180578A4
:10021000401C6B075B0F01D10378401C2A1106D1EB
:100220000278401C03E006780E70401C491C5B1EDF
:10023000F9D12B0705D40023521E0DD40B70491C95
:10024000FAE70378401CCB1A921C03E01D780D706E
:10025000491C5B1C521EF9D5A142D8D3002070BDA9
:1002600010B5084C0421204600F056F8012804D1AE
:10027000204600F040F8044908800421204600F0A0
:1002800008F810BD00240140000000208162426196
:100290007047016070470029816801D0012200E0A9
:1002A0000222114381607047064910B5884208D187
:1002B00044150121204600F04DFD0021204600F0AC
:1002C00049FD10BD00240140826800210123DB07A5
:1002D0001A4382600F231B038268491CD20FD20786
:1002E000994201D0002AF7D18168002901DB006C16
:1002F000704700207047006C80B2704702460020B3
:10030000CB0104D5926801231B069A4300E01268D2
:100310000A4200D00120704702465368002012684C
:100320000B400A4202D0002B00D001207047002A67
:10033000426801D00A4300E08A43426070470000EF
:1003400030B5C268074B8C681A404B680D78234360
:10035000CC686D032C43096923430B431343C360EB
:1003600030BD000000D2FFFF81680422114381608C
:1003700070470021017041608160C1600161704778
:100380003EB50121080500F0C1FC042000900320C7
:100390006946087101244C71064800F0F4F800F039
:1003A0000BF80C20694608704C708C70684600F0A1
:1003B00083FC3EBD000C004810B5012186B0480208
:1003C00000F0BCFC164C2046FFF76EFF6846FFF7B6
:1003D000D0FF012069460870002102910391049129
:1003E00069462046FFF7ACFF072210212046FFF7A1
:1003F0004DFF2046FFF768FF012204212046FFF74A
:1004000096FF01212046FFF746FF01212046FFF716
:1004100075FF0028F9D02046FFF7A6FF06B010BDF3
:10042000002401403EB51120694608700120487043
:100430008870684600F040FC0121102000F072FC3A
:100440000B4801901F2069460A4C0880204600F0A6
:1004500071FE0121204600F043FE01221146204694
:1004600000F05EFE0121204600F042FE3EBD00008D
:10047000E703000000100040F0B50B2706463F04DC
:10048000384600F06FF8042811D1094C206B022582
:1004900028432063064840384661016940221143E1
:1004A0000161384600F05EF8216BA9432163F0BD7D
:1004B00040200240F0B507460B200E46000400F035
:1004C00051F804280CD1074C206B042528432063E5
:1004D0003E700B20000400F045F8216BA943216316
:1004E000F0BD00004020024070B50D46044600F00B
:1004F00029F80320800620180446FFF7BDFF29468F
:100500002046FFF7D7FF00F015F870BD03229206D2
:10051000801800780870704705490420CA68D2071F
:1005200001D001207047C968C906FBD50220704779
:100530000020024002480169802211430161704796
:100540000020024004480169090603D503494160BF
:1005500003494160704700000020024023016745C5
:10056000AB89EFCD00B50346FFF7D6FF02E0FFF7FA
:10057000D3FF5B1E012803D0002B00D1052000BD56
:10058000002BF4D1FAE7F0B50022032501230C6813
:1005900093401C409C422BD10C79012C01D0022CA1
:1005A00013D1876854002E46A640B74387604E7922
:1005B000A64084682643866044689C434460436840
:1005C0008C799440A4B223434360066853002C46C0
:1005D0009C40A64306600E7907689E403E43066035
:1005E000C668A643C660CC799C40C3681C43C460FF
:1005F000521C102ACAD30A7A002A026B096802D058
:100600008A430263F0BD0A43FBE74B07DB0E9A40C7
:10061000C90810B589000818016A0F249C40A1433D
:100620000162016A1143016210BDFFB583B00D463E
:100630000F201E461446012140040C9F00F066FB6B
:10064000694600950C718F71CE71012048710020B0
:1006500008720398FFF797FF07B0F0BDFEE70000B0
:10066000FFB5284F81B01026BE62274D4024AC62F2
:100670002A2000F03FFCAC61BE61AC620198801C96
:1006800000900004000E00F035FC0098C0B200F0AD
:1006900031FCAC61AC620398801C00900004000E39
:1006A00000F028FC0098C0B200F024FCAC61BE62EF
:1006B000AC622B2000F01EFCAC61BE61AC62029803
:1006C000433000900004000E00F014FC0098C0B20B
:1006D00000F010FCAC61AC62049843300090000460
:1006E000000E00F007FC0098C0B200F003FCAC6103
:1006F000BE62AC622C2000F0FDFBAC61BE6105B0B7
:10070000F0BD00000004004800080048FFB581B0BB
:1007100004980D46401E83B20398401E82B2019891
:10072000FFF79EFF0A984026000A0D4F009011E047
:10073000019C0AE0BE62009800F0DCFB0A98C0B29F
:1007400000F0D8FBBE61641CA4B203988442F1D3CC
:100750006D1CADB204988542EAD305B0F0BD00002F
:1007600000080048F8B50024FD4F234601228021EF
:1007700038460094FFF759FF0023012240213846F4
:100780000094FFF752FFF74D002301221021284665
:100790000094FFF74AFF1026AE618022BA61F24C46
:1007A0000021002000BF401CA042FBDB491C0529A2
:1007B000F7DBBA620021002000BF401CA042FBDB37
:1007C000491C0529F7DBBA610021002000BF401C4D
:1007D000A042FBDB491C1429F7DBAE624020B86263
:1007E000012000F087FB4020B861AE6100210020AD
:1007F00000BF401CA042FBDB491C1429F7DBAE62A2
:100800004020B862112000F075FB4020B861AE6155
:100810000021002000BFD44A401C9042FADB491C52
:100820003229F6DBAE624024BC62B12000F062FBEC
:10083000BC61AE61BC62022000F05CFBBC61BC62CA
:10084000352000F057FBBC61BC62362000F052FB43
:10085000BC61AE62BC62B22000F04CFBBC61AE6118
:10086000BC62022000F046FBBC61BC62352000F097
:1008700041FBBC61BC62362000F03CFBBC61AE6257
:10088000BC62B32000F036FBBC61AE61BC620220EA
:1008900000F030FBBC61BC62352000F02BFBBC617A
:1008A000BC62362000F026FBBC61BC62022000F076
:1008B00021FBBC61BC62352000F01CFBBC61BC624A
:1008C000362000F017FBBC61AE62BC62B42000F0C1
:1008D00011FBBC61AE61BC62032000F00BFBBC618C
:1008E000AE62BC62C02000F005FBBC61AE61BC62C0
:1008F000A22000F0FFFABC61BC62022000F0FAFA0C
:10090000BC61BC62842000F0F5FABC61AE62BC62DE
:10091000C12000F0EFFABC61AE61BC62C52000F0FE
:10092000E9FABC61AE62BC62C22000F0E3FABC61CD
:10093000AE61BC620D2000F0DDFABC61BC6200203B
:1009400000F0D8FABC61AE62BC62C32000F0D2FAFB
:10095000BC61AE61BC628D2000F0CCFABC61BC62AF
:100960002A2000F0C7FABC61AE62BC62C42000F06D
:10097000C1FABC61AE61BC628D2000F0BBFABC6103
:10098000BC62EE2000F0B6FABC61AE62BC62C5206B
:1009900000F0B0FABC61AE61BC620A2000F0AAFAB5
:1009A000BC61AE62BC62362000F0A4FABC61AE61EC
:1009B000BC62C82000F09EFABC61AE62BC62E0205E
:1009C00000F098FABC61AE61BC62122000F092FAAD
:1009D000BC61BC621C2000F08DFABC61BC621020BE
:1009E00000F088FABC61BC62182000F083FABC6198
:1009F000BC62332000F07EFABC61BC622C2000F0A7
:100A000079FABC61BC62252000F074FABC61BC625A
:100A1000282000F06FFABC61BC62282000F06AFA5E
:100A2000BC61BC62272000F065FABC61BC622F206B
:100A300000F060FABC61BC623C2000F05BFABC6173
:100A4000BC62002000F056FABC61BC62032000F0DA
:100A500051FABC61BC62032000F04CFABC61BC627C
:100A6000102000F047FABC61AE62BC62E12000F0E9
:100A700041FABC61AE61BC62122000F03BFABC617D
:100A8000BC621C2000F036FABC61BC62102000F091
:100A900031FABC61BC62182000F02CFABC61BC6267
:100AA0002D2000F027FABC61BC62282000F022FA59
:100AB000BC61BC62232000F01DFABC61BC6228202E
:100AC00000F018FABC61BC62282000F013FABC6187
:100AD000BC62262000F00EFABC61BC622F2000F040
:100AE00009FABC61BC623B2000F004FABC61BC6244
:100AF000002000F0FFF9BC61BC62032000F0FAF9AD
:100B0000BC61BC62032000F0F5F9BC61BC6210203E
:100B100000F0F0F9BC61AE62BC623A2000F0EAF984
:100B2000BC61AE61BC62052000F0E4F9BC61AE625C
:100B3000BC62292000F0DEF9BC61AE610A4A0021E6
:100B4000002000BF401C9042FBDB491C3229F7DB30
:100B500000204023802201460090FFF7D7FDF8BD1A
:100B60000008004800040048881300000F2801D83E
:100B7000032901D90120704709010818014908809B
:100B800000207047A0010020F8B5203AD4B20A46F0
:100B90001F460F3293B2C21D92B289B280B2FFF7E4
:100BA0005FFD15490026200140180090855D002456
:100BB000280609D51149402088620698000A00F0ED
:100BC00099F90698C0B206E00C4940208862380ABC
:100BD00000F090F9F8B200F08DF9084940208861E2
:100BE0006804050C641C082CE2DB761C102E01DA6C
:100BF0000098DBE7F8BD0000901D000800080048E1
:100C0000F7B507461A4801880807090909010A4685
:100C10000F32400E93B2C21DFFF722FD00263D7831
:100C20000024280608D51349402088620298000A4B
:100C300000F060F9029807E00E49402088620198B0
:100C4000000A00F057F90198C0B200F053F90949C1
:100C5000402088616806050E641C082CE1DB761CC8
:100C60007F1C102EDBDB02490888401C0880FEBD7B
:100C7000A001002000080048F8B516460F460446BB
:100C80000B4D10E029883F2901D90120F8BD080744
:100C90000909400E09013B460096FFF775FF2888B9
:100CA000401C2880641C2278002AEBD10020F8BD6B
:100CB000A00100207047000030B58278012401783F
:100CC000002A15D08B080E4A9B009A1813688907D2
:100CD000C90EFF258D40AB434578AD072D0E8D40E5
:100CE0001D4315600078C006C00E8440054804E02E
:100CF000C806C00E844003488030046030BD000048
:100D000000E400E000E100E070470000044A002930
:100D1000516901D0014300E08143516170470000F7
:100D200000100240044A0029D16901D0014300E0CB
:100D30008143D1617047000000100240044A00293D
:100D4000916901D0014300E0814391617047000047
:100D500000100240044A0029D16801D0014300E09C
:100D60008143D1607047000000100240F8B52C4963
:100D7000044648680C222B4E104003D0042801D0B2
:100D80000C281FD0264D2660686837460006000FE5
:100D900041002548415A3846FFF7ACF96060696860
:100DA000214A4905490F083A515CC8400546A060F0
:100DB0001E480169890F09D00169890F01290FD0E7
:100DC000680812E07D2080022060DBE71448C03014
:100DD000806A4000C10E1648891CFFF78BF904E0B9
:100DE0000069800F022801D0A808E0600C48016B60
:100DF000C90601D4266100E02761016B89070AD08A
:100E0000016B8907890F012907D0006BC043800758
:100E100000D16661F8BD6561F8BD6761F8BD00008D
:100E2000001002400048E801701D00080024014045
:100E30000090D0030029016802D04022114301E054
:100E4000014A114001607047BFFF0000F0B5012169
:100E50000D0387B02846FFF771FF0024224E23467A
:100E60000222102130460094FFF7DFFB002302220C
:100E7000082130460094FFF7D8FB1C4F00230222C4
:100E8000102138460094FFF7D0FB0222042130469F
:100E9000FFF7BBFB022203213046FFF7B6FB02221D
:100EA00004213846FFF7B1FB6946FF208C800530EE
:100EB000C8800720000208814C818C81E810C8811D
:100EC000182008824C8207208882094C01A92046FC
:100ED00000F01EF82946204600F046F80121204681
:100EE000FFF7A8FF07B0F0BD000C00480004004861
:100EF0000030014010B5054C0146204600F03EF898
:100F0000A0680006FCD4002010BD000000300140A5
:100F100030B50268CC8993B2C122920113400A888D
:100F20000D892243CC882C4322434C8922438C894F
:100F300022431A4302604268094B92B21A408B88DE
:100F4000134343600A8A02610268042392B249880B
:100F50009A4311430160C169024A1140C16130BD29
:100F6000FFF00000FFF700004268034B1A404260A8
:100F700042680A4342607047FFEF00000173704708
:100F80007047000030B585B00023244800930193DA
:100F900002930393049301680124214301601F49D4
:100FA000C0318A6A0F25ED02AA438A628A6A072540
:100FB000ED022A438A621A4D022102680A40019218
:100FC000009A521C0092019A002A02D1009AAA4269
:100FD000F3D1026892071ED5124A01941368DB0808
:100FE000DB0002930B4313604168F02291430391AD
:100FF00041604168072212029143049141604168B7
:101000008908890041604168416041680907890F8A
:10101000FBD105B030BD0193FBE70000001002409A
:10102000FFFF0000002002407047000010B512488A
:1010300001680122114301604168104A114041607A
:10104000016B132291430163002484600C49096AF7
:101050000A0C89B20A4209D10268CA064905120E71
:10106000890E09020A43016811430160FFF78AFFF4
:101070000448446310BD0000001002401CB8FFF893
:1010800000F8FF1F4020024010B5084808220378EE
:101090000749002B02D08A61002101E08A62012108
:1010A00001700121880700F01FF810BDA201002087
:1010B0000008004810B5084C0121204600F024F833
:1010C000002807D005494A68521C4A600121204681
:1010D00000F00AF810BD00000010004000000020E1
:1010E000C94389B201617047C94389B20161704740
:1010F0000029016802D00122114301E0014A114098
:1011000001607047FEFF0000024613690020D268AC
:101110000B400A40002B02D0002A00D0012070476B
:10112000002AC26801D00A4302E0C94389B20A40DA
:10113000C260704710B502680F4B92B2984203D05C
:101140000124A407A04203D17024A2434C88224367
:101150000A4CA04203D00A4C22400C892243026070
:101160004A68C2620A888262984201D1897A016320
:101170000121416110BD0000002C01400010004021
:10118000FFFC00000029016802D00122114301E0A8
:101190004908490001607047F0B509208BB0012172
:1011A0004004FFF7B3FD01218803FFF7C7FD0927BE
:1011B000FF06012203213846FFF727FA0122062104
:1011C0001B48FFF722FA08200090022669460E719C
:1011D00001254D7100248C71CC713846FFF7D3F98D
:1011E0004020009069460E711148FFF7CCF9E120CC
:1011F0000994400205940694079404900C200D4C29
:10120000089004A9204600F02FF81B2069460873B7
:101210004D738D7303A8FFF74FFD01220649204649
:1012200000F00CF801212046FFF7ACFF0BB0F0BD39
:10123000000C0048003801400501050010B50B0402
:101240001C0E01238B40022C02D0032C02D002E0A2
:10125000001D00E008300168002A01D0194300E0B9
:101260009943016010BD000030B50446006887B0A6
:101270000D46400840002060606803210903884350
:10128000A9680143616020681849EA6808406968F4
:1012900011432A69024311432160A0680321090216
:1012A000884369690143A1606846FFF75FFD104804
:1012B000844201D1059800E0029821680904296858
:1012C00000D54000FEF716FF2A6852088A4200D86F
:1012D000401C2168090404D50107064A490F104043
:1012E000084380B2E06007B030BD0000F3E9FFFFC3
:1012F00000380140F0FF00000FB410B504A9074BFF
:1013000002AA039800F01CF8044602A9002000F08D
:1013100051FA204610BC08BC04B01847B5170008A5
:1013200002E008C8121F08C1002AFAD170477047AE
:10133000002001E001C1121F002AFBD1704700000C
:10134000FFB591B00F460546002606E025280AD0D5
:10135000149A139990476D1C761C28780028F5D1B3
:10136000304615B0F0BD002400940121F34A0294E8
:1013700000E004436D1C2B780846203B9840104247
:10138000F7D128782A280ED0022228780146303951
:10139000092915D800990A235943303940181443B4
:1013A0006D1C0090F1E701CF0090002805DA0120C4
:1013B00040030443009840420090022004436D1C07
:1013C00028782E2815D10420044368786D1C2A281B
:1013D0000AD101CF6D1C02900BE002990A22514301
:1013E000303940186D1C029028780146303909299F
:1013F000F3D928786C2810D006DC4C281AD068283D
:101400000ED06A2817D104E0742813D07A2812D19C
:1014100010E00120400504430CE00121090501E032
:10142000032109050C436978814203D1012000059D
:1014300024186D1C6D1C28786E281ED00CDC6328C7
:1014400031D004DC00288BD0582811D1B2E06428B8
:101450007BD069280CD178E073282DD004DC6F286C
:1014600070D0702804D1A7E075286CD078286BD094
:10147000149A13999047761C62E06002400F02288C
:1014800007D003280AD0042838680AD006603F1D18
:1014900056E03868F11706604160F8E73868068062
:1014A000F5E70670F3E73878694608740020487459
:1014B00004A80390012003E0386803900020C04393
:1014C0003F1D61070FD5002101E00199491C029AD7
:1014D0000191914213DA8142F7DB019A0399895C09
:1014E0000029F2D10BE0002101E00199491C019192
:1014F0008142FADB019A0399895C0029F5D10199AF
:101500000098139A401A00902146149B00F03CF971
:1015100001998019461807E0039803990078491C3F
:101520000391149A139990470198401E0190401C12
:10153000F2D12146149B139A009800F015F98619F0
:101540006D1C0AE741E033E034E00A2000210490FA
:1015500005916002410F022905D001CFC2179446C0
:10156000032905D007E0FF1DFF08FF0003CF06E0B9
:1015700000B2C2179446042902D140B2C1178C466A
:1015800000226146944506DA0A4600214042914114
:101590008C462D2102E0210504D52B216A461176C7
:1015A000012103E0E10701D02021F7E7019155E097
:1015B0000A200BE0102009E01020049000210420F4
:1015C000044308200591029003E0082000210591C2
:1015D00004906002410F022905D001CF00229446F9
:1015E000032906D006E0FF1DFF08FF0003CF8C464D
:1015F00003E080B2042900D1C0B20021019121078B
:101600002CD529780391702906D0049A1021059BC6
:101610004A401A4305D00EE040216A461176012166
:1016200008E06146014306D030216A4611760399ED
:10163000517602210191049A0821059B4A401A43E0
:101640000CD16146014301D1610707D530216A46BB
:101650001176012101910299491E02912978582998
:1016600004D037A103910FA90F910DE039A1F9E73B
:101670006146059B049AFEF765FD039B8C469B5CC7
:101680000F9A521E0F92137061460143F0D10F98CA
:1016900007A9081A20300390600704D50120000430
:1016A0008443029801E0012002900399884201DD01
:1016B000401A00E000204118029001980918009893
:1016C000401A0090E00306D42146149B139A009818
:1016D00000F05AF886190020049008E006A9085C7A
:1016E000149A139990470498401C761C0490019911
:1016F0008842F3DBE0030CD52146149B139A009833
:1017000000F042F8861904E0149A302013999047AB
:10171000761C0299481E02900029F5DC08E00F981B
:101720000F990078491C0F91149A13999047761CD1
:101730000399481E03900029F1DCFAE6092801000C
:101740003031323334353637383961626364656637
:1017500000000000303132333435363738394142F9
:101760004344454600000000F8B5044600251E46E7
:101770001746880404D405E039462020B0476D1C84
:10178000641EF9D52846F8BDFFB50446002581B092
:101790001E46C80301D5302700E02027880404D561
:1017A00005E038460399B0476D1C641EF9D52846FC
:1017B00005B0F0BD0A68531C0B6010707047000044
:1017C00070B5184A184CD16801250023E06800293B
:1017D0001BD0012918D101281DD01069012813D16F
:1017E000114910481431CC680078012C17D02831E9
:1017F000CC68012C08D1401CCB60C1B21170002014
:10180000FEF772FE00F0DCF870BD0128FCD1E36049
:10181000D560156170BDE3601561D360E0E7401EDF
:10182000CB60EAE7080000205001002010B5044614
:101830002169406888470006000E04D0002020601F
:10184000A060E06010BD20680028FBD1A0681E28C1
:1018500002DA401CA06010BD0120E060206010BDD5
:1018600010B50848FFF7E2FF06481430FFF7DEFF27
:1018700004482830FFF7DAFF02483C30FFF7D6FF74
:1018800010BD0000500100200C49012807D002289B
:1018900008D0032809D004280AD00120704708691D
:1018A000800608E00869C00605E00869000702E054
:1018B000034800698007C00F704700000008004817
:1018C000000C004808B5FFF7C1FAFFF765FCFEF70A
:1018D00049FF00210846FFF749F9214A002121A0CC
:1018E000FFF7CAF9002009240346E406009001220C
:1018F00002212046FEF799FE0221A162FEF792FD29
:10190000FEF73EFD1B490020FEF700FE01241A4DA4
:1019100023460022202128460094FEF786FE01235C
:101920000022102128460094FEF77FFE01230022AA
:10193000082128460094FEF778FE012300220221A8
:101940000E480094FEF771FE0D4D0A4C2868A169FF
:101950008842FBD000F0B0F8A069401CA061F5E718
:10196000FFFF000052616262697420436F6F6C6513
:10197000720000000800002000080048000C004829
:101980000400002010B500210846FFF7EFF8064AD2
:10199000002106A0FFF770F900F072F900F0ACF832
:1019A00000F030F910BD0000FFFF000052616262DC
:1019B000697420436F6F6C65722020200000000066
:1019C00030B585B014216846FEF7B1FB2F4D30A12C
:1019D0002A786846FFF790FC00210846FFF7C6F812
:1019E00028692F4C01283ED0224601283DD00021F5
:1019F0006846FFF741F92869012838D022460128B6
:101A000037D0002121481C30FFF7FAF801210020CF
:101A1000FFF7ACF8286902282DD0224602282CD0E6
:101A2000002120A0FFF728F902210020FFF79EF8EF
:101A30002869032823D02246032822D0002119A098
:101A4000FFF71AF903210020FFF790F8286904280E
:101A500019D02246042800D00024214611A0FFF707
:101A60000BF905B030BD0022BFE72146C0E70022D8
:101A7000C5E72146C6E70022D0E72146D1E700228C
:101A8000DAE72146DBE70022E4E700000800002057
:101A90007461726765742074656D703A25336400F3
:101AA000FFFF0000202020202020202020202020B8
:101AB000202020200000000010B50E4C7D21C90020
:101AC0006069FEF717FB00290CD1E068002802D0FE
:101AD000012803D004E0FFF755FF01E0FFF770FF96
:101AE00000F02AF9FFF7BCFEFFF76AFE6069401CB0
:101AF000606110BD08000020F0B587B0142101A876
:101B0000FEF715FB2E4800882E4A2F4D1188814282
:101B100001D22EA204E02F49098B81420FD92EA2B7
:101B200030A101A8FFF7E8FB02210020FFF71EF813
:101B30002A46002101A8FFF79FF807B0F0BD002456
:101B40006100535A834203D389184988814202D3E2
:101B5000641C8D2CF4DB6100535A7D26F600891835
:101B60007343498870437143181A6422591A5043C9
:101B7000FEF7C0FA134E07462C3E70682018143842
:101B800000F0A6F80A213846FEF7B4FA03460091A1
:101B9000706817A1221801A8143AFFF7ADFB0221C3
:101BA0000020FEF7E3FF2A46002101A8FFF764F8B2
:101BB00030462A4600211C30FFF722F8BDE700001E
:101BC0000000002034000020FFFF0000746F6F2031
:101BD0006C6F770034010020746F6F20686967684C
:101BE0000000000074656D70206572723A25730004
:101BF00074656D703A202020202533642E256425DD
:101C00006400000030B585B014216846FEF78FFAF5
:101C100003210020FEF7AAFF114C12A1227868468A
:101C2000FFF76AFB114D00212A466846FFF724F8AA
:101C300020462A4600211C30FEF7E2FFA06800285B
:101C400001D00BA200E00BA20BA16846FFF754FBEA
:101C50002A4600216846FFF70FF805B030BD0000A6
:101C6000080000207461723A25336400FFFF000011
:101C7000204F4E004F464600202073773A257300D0
:101C800000B587B0142101A8FEF751FA09480AA14E
:101C90000CC80068009001A8FFF72EFB012100206E
:101CA000FEF764FF094A002101A8FEF7E5FF07B02F
:101CB00000BD0000A401002072756E3A2020202093
:101CC0002532643A2532643A25326400FFFF000071
:101CD000F0B5184A164D174C2E78936851680227B4
:101CE00012680C34B04213DB0120A8600920C00642
:101CF00087610F31A360226061603C2907DB521CC1
:101D00003C3922606160182A01D100202060F0BDBA
:101D100020689042FBD160688842F8D1A068984260
:101D2000F5D10020A8600920C0068762F0BD000040
:101D300008000020A40100200A498868401C88602F
:101D40003C280DD148680022401C8A6048603C282D
:101D500006D14A600868401C0860182800D10A6053
:101D600070470000A40100200000000001020304ED
:101D70000100060001000100010001000100010056
:101D80000200040008001000400080000001000272
:101D90000000000000000000000000000000000043
:101DA000000000001818181010000018180000009B
:101DB000000000007E6624240000000000000000F7
:101DC0000000000024247E24247E2424000000003F
:101DD0000000000008083E203E023E080800000007
:101DE0000000000060620408181020460600000091
:101DF000000000000038444428304A443A00000003
:101E0000000000001818181010000000000000006A
:101E1000000000000408101010101008040000005A
:101E2000000000002010080808080810200000002A
:101E30000000000000082A1C081C2A0800000000FE
:101E400000000000000008083E0808000000000034
:101E50000000000000000000001C0404040000005A
:101E60000000000000000000007E000000000000F4
:101E70000000000000000000000018180000000032
:101E800000000000020204080810202040000000AA
:101E9000000000007E424242424242427E00000078
:101EA0000000000038080808080A0A0A3E0000007E
:101EB000000000007E0202027E4040407E000000E2
:101EC000000000007E0202023C0202027E000000CE
:101ED0000000000020222222223F02020200000015
:101EE000000000003E2020203E0202423E00000092
:101EF0000000000060404040407E42427E00000002
:101F0000000000007C040404081010101000000001
:101F1000000000003C2424247E4242427E00000057
:101F2000000000007E42427E020202020600000023
:101F30000000000000181800001818000000000041
:101F400000000000003030000038080808000000E1
:101F50000000000000020C3040300C0200000000C5
:101F60000000000000007E007E0000000000000075
:101F7000000000000040300C020C30400000000067
:101F8000000000000C12224C102020002000000055
:101F9000000000003C420232525252522C0000001B
:101FA000000000001818182424243C4242000000BD
:101FB000000000007C4242427C4242427C00000021
:101FC000000000001E202040404020201E00000095
:101FD000000000007824242222222424780000001B
:101FE000000000007E404040784040407E000000FD
:101FF000000000007E40407C404040404000000027
:10200000000000001E202040404E42423C000000E4
:1020100000000000424242427E4242424200000032
:10202000000000007C101010101010107C00000048
:102030000000000002020202022222221C00000014
:1020400000000000424448506050484442000000F4
:102050000000000040404040404040407E00000002
:1020600000000000C6C6AA9282828282820000001E
:102070000000000062625252524A4A464600000086
:1020800000000000182424424242242418000000CA
:10209000000000007C424242427C40404000000080
:1020A000000000000E12224242525C487E000000F6
:1020B000000000007C42427C48484442420000004C
:1020C000000000003C422010100804423C000000C8
:1020D000000000003E2A0808080808080800000060
:1020E0000000000042424242424242423C000000A4
:1020F0000000000042424242242418181800000048
:102100000000000044444454545454542800000037
:102110000000000042242418081824244200000073
:10212000000000002222221408080808080000000D
:10213000000000007E040408101020207E00000033
:10214000000000007E505050505050507E00000063
:102150000000000020201008080402020100000016
:10216000000000007E0A0A0A0A0A0A0A7E0000002D
:10217000000000000018183C246642000000000027
:102180000000000000000000000000000000FF0050
:102190000000001804000000000000000000000023
:1021A0000000000000003C02023E42463A000000EF
:1021B0000000000040405C62424242625C0000005D
:1021C0000000000000001E60404040601E00000053
:1021D0000000000002023A46424242463A00000035
:1021E0000000000000003C42427E40403E000000F3
:1021F000000000000E103C10101010101000000025
:102200000000000000003A464242463A02027C00CA
:102210000000000040405C62424242424200000036
:102220000000001818003808080808083E000000E0
:102230000000000606001E020202020202221C002A
:1022400000000000404044485060504C42000000F4
:102250000000000038080808080808083E000000D0
:10226000000000000000685454545454540000000E
:102270000000000000005C62424242424200000056
:102280000000000000003C42424242423C0000008C
:102290000000000000005864424242645840400080
:1022A0000000000000003A46424242463A02020064
:1022B0000000000000005C6242404040400000001E
:1022C0000000000000003E40300C02027C000000D4
:1022D0000000000020207C20202020221C00000084
:1022E0000000000000004242424242463A00000024
:1022F00000000000000042424224241818000000A0
:102300000000000000008282929292AA4400000025
:1023100000000000000042241818182442000000A9
:1023200000000000000042424224241808107000FF
:102330000000000000007E02041820407E00000023
:102340000000000006080808300808080600000021
:102350000000000008080808080808080800000035
:1023600000000000300808080608080830000000D7
:1023700000000000000000001A2C00000000000017
:10238000A023000800000020A40100000A020008A9
:10239000E4240008A40100203C01000030130008E0
:1023A0008132320516FBFFFFFF147050703B1E2078
:1023B00001221E105B790E660E4C0E380E1E0E06A4
:1023C0000EEC0DD60DB60D9C0D800D600D3D0D244F
:1023D0000D090DE90CC80CA50C810C5D0C390C1312
:1023E0000CED0BC50B9E0B750B4C0B220BF80ACD9D
:1023F0000AA20A710A490A1E0AF009C30996096964
:10240000093C090E09E008B3088508580828081097
:102410001808D007A50779074D072107F706CD064D
:10242000A2067906500628061081067406B2058CAD
:1024300005670543051F05FC04DA04B80497047713
:1024400004580439041B04FE03E103C503AA038FE7
:102450000375035C0344032C031503FE02E802D357
:1024600002BE02AA029602830271025F024E023D80
:10247000022C021C020D02FE01EF01E101D401C693
:1024800001B901AD01A10195018A017F01740169C2
:10249000015F0155014C0143013A0131012901213C
:1024A00001190112010A010301FC12F612EF12E8F0
:1024B00012E212DC12D712D112CB12C612C112BC18
:1024C00012B712B312AE12AA12A512A1129D7299DE
:1024D000B20113891842080A1104140A1103140ADC
:0424E00011021400D1
:04000005080000C12E
:00000001FF
